:100000000C948A000C94A5000C94A5000C94A500F7
:100010000C94A5000C94A5000C94A5000C94A500CC
:100020000C94A5000C94A5000C94A5000C94A500BC
:100030000C94A5000C94A5000C94A5000C94A500AC
:100040000C94A5000C94A5000C9493050C94BD058C
:100050000C94A5000C9404040C94A5000C94A50029
:100060000C94A5000C94A5000C94A5000C94A5007C
:100070000C94A5000C94A5000C9443060C946F06F8
:100080000C94A5000C94A5000C94A500427566661E
:100090006572204F766572666C6F77204572726F5D
:1000A000723A200055415254204F76657272756E37
:1000B000204572726F723A200055415254204672A8
:1000C000616D65204572726F723A2000554152543D
:1000D0003020427566666572204F766572666C6F79
:1000E00077204572726F723A200055415254302089
:1000F0004F76657272756E204572726F723A20008B
:100100005541525430204672616D65204572726FC0
:10011000723A200011241FBECFEFD0E1DEBFCDBF69
:1001200013E0A0E0B1E0E4E2FCE102C005900D9232
:10013000AC3FB107D9F716E0ACEFB3E001C01D92B8
:10014000AE32B107E1F70C94C8000C94000020E037
:1001500030E00BC0000000000000000000000000C4
:100160000000000000002F5F3F4F2817390791F76C
:100170000895CF93DF93C0E0D0E08FEF90E00E942E
:10018000A7002196CF33D105C1F7DF91CF91089514
:100190006F927F928F929F92AF92BF92CF92DF9297
:1001A000EF92FF920F931F93CF93DF9310920A0663
:1001B0001092090610922706109226061092140635
:1001C0001092130610921A061092190610922B061E
:1001D00010922A068FEF9FE790930E0680930D06EC
:1001E00080E190E09093100680930F060E941B0719
:1001F00087E690E00E94E20587E690E00E9499067B
:1002000082B1806F82B983B1806F83B98FEC86B978
:100210007894C0E0D0E0F5C28FEF90E00E94A70094
:100220000F5F1F4F0F3F1105B9F72196C830D10559
:1002300009F0E7C280E091E00E94E60688E191E0E3
:100240000E94E6068BE491E00E94E60689E691E0D2
:100250000E94E60689E891E00E94E60680EB91E0C4
:100260000E94E60689EC91E00E94E60684EE91E0A9
:100270000E94E6068FE092E00E94E606AA24BB24D4
:1002800088249924662477241C980E94B90083B19D
:10029000806F83B91D980E94B90083B1806F83B9C4
:1002A0001E980E94B90083B1806F83B91F980E9485
:1002B000B90083B1806F83B98AE492E00E94E606B8
:1002C0008091280690912906892B19F4AA24BB2431
:1002D00084C080E190E09093100680930F06009117
:1002E00017061091180602541E40B801882777FDA2
:1002F0008095982F0E94B30A17FF06C020E030E0D7
:1003000040E857E40E9432092AE735EA41E55CE318
:100310000E945F090E94AE076B017C017093160674
:100320006093150600910706109108060C561C40B4
:10033000B801882777FD8095982F0E94B30A17FF90
:1003400006C020E030E040E857E40E94320923E78D
:1003500035EA49EF5BE30E945F090E94AE07DC01CA
:10036000CB01909325068093240664E670E00E94FA
:10037000C70D9B01220F331F260F371FC60164E6EE
:1003800070E00E94C70D6F5F7F4F260F371F2770E9
:1003900030702A153B0511F059011DC00894811CCD
:1003A000911C89E288169104C0F0A614B70461F08C
:1003B00083E592E00E94E6068A2D805D0E94D006C9
:1003C0008AE592E00E94E60610922B0610922A0619
:1003D0003501AA24BB24882499240E94FB058C01A2
:1003E00090FD48C093FF04C080E091E00E94F306B6
:1003F00012FF04C08AEE90E00E94F30611FF04C0D1
:100400008CEC90E00E94F3060C34110549F4109234
:100410001A06109219068DE592E00E94E6062AC09F
:100420000134110539F580912A0690912B06892B0C
:1004300009F581E090E090932B0680932A068FEFD8
:100440000E94160681E00E94160680E00E941606B1
:1004500087E00E94160680E00E94160681E00E9456
:10046000160689E00E94160684E090E0909310063C
:1004700080930F060E94B506EC0190FD05CF93FF17
:1004800004C089EB90E00E94F306D2FF04C084EA26
:1004900090E00E94F306D1FF04C08CE890E00E9437
:1004A000F306C335D10509F043C087E792E00E9407
:1004B000E60682E090E090930C0680930B0686E0BF
:1004C00090E090932D0680932C0666E082E00E94D7
:1004D000830783E090E090930C0680930B06909343
:1004E0002D0680932C0663E083E00E94830784E05E
:1004F00090E090930C0680930B0610922D061092BC
:100500002C0660E084E00E94830785E090E09093F1
:100510000C0680930B0610922D0610922C0660E0BC
:1005200085E00E94830787E892E00E94E6062BC0E0
:10053000C235D10539F481E992E00E94E6060E94B5
:1005400036072EC0C435D105C9F482EA92E00E9474
:10055000E6068EEA92E00E94280683E193E00E947C
:1005600028068EEA92E00E94E60683E193E00E946C
:10057000E6068AE493E00E94E6062BC0CC34D1055F
:1005800011F48CE469C0C134D10551F481E40E94B6
:10059000160682E090E09093100680930F0675C0D7
:1005A000CD34D105B1F48FEF0E94160681E00E9490
:1005B000160680E00E94160687E00E94160680E07C
:1005C0000E9416068FE50E94160687E60E94160610
:1005D00073C020E030E0CE01C197029710F421E013
:1005E00030E080E090E0C533D10511F481E090E087
:1005F000282B392B40E050E0C433D10511F441E001
:1006000050E080E090E0C333D10511F481E090E048
:10061000842B952B40E050E0C633D10511F441E026
:1006200050E0842B952B282B392B232BB9F08FEFFF
:100630000E94160681E00E94160680E00E941606BF
:1006400083E00E94160680E00E9416068C2F8053DD
:100650000E9416068C2F8C520E941606CD32D105B0
:10066000A1F48FEF0E94160681E00E94160681E039
:100670000E94160680E00E94160680E00E94160680
:1006800080E00E94160682E096C0CB32D105A1F42C
:100690008FEF0E94160681E00E94160680E00E94FD
:1006A000160680E80E94160680E00E94160680E08A
:1006B0000E94160681E87FC010E0C537D10509F415
:1006C00011E0FF24C436D10511F481E0F82E812F0A
:1006D0008F29992720E030E0C936D10511F421E0B7
:1006E00030E0822B932B40E050E0C237D10511F46B
:1006F00041E050E020E030E0CC36D10511F421E0BB
:1007000030E0242B352B40E050E0CF36D10511F4FA
:1007100041E050E0242B352B822B932B892B09F4BD
:100720004CC080E190E09093100680930F068FEF0D
:100730000E94160681E00E94160680E00E941606BE
:10074000112319F400E010E005C088E00E941606AD
:1007500009E410E0FF2029F080E10E94160601E57F
:1007600010E0CC36D10531F484E00E94160605E491
:1007700010E01AC0C237D10531F482E00E9416069B
:1007800003E410E011C0C936D10531F480E20E94C3
:10079000160601E610E008C0CF36D10529F480E442
:1007A0000E94160601E810E080E20E94160680E230
:1007B0000E941606802F0E941606C0E0D0E08FEF40
:1007C00090E00E94A7002196CF3FD105C1F78FEF9F
:1007D0000E94160681E00E94160680E00E9416061E
:1007E00080E00E94160680E00E94160680E00E94CB
:1007F000160681E00E94160681E693E00E94E60656
:1008000043CD00E010E008CD1F920F920FB60F927B
:1008100011240F931F932F933F934F935F936F93E5
:100820007F938F939F93AF93BF93EF93FF938091A9
:100830000D0690910E06019790930E0680930D067B
:100840002FE38F3F920709F464C0892B09F061C040
:100850008FEF9FE790930E0680930D0680910F0611
:100860009091100601979093100680930F062091A7
:10087000190630911A062F5F3F4F30931A062093C6
:100880001906892B31F480E190E090931006809353
:100890000F062830310520F087E793E00E94E60636
:1008A0000091130610911406B801882777FD8095F2
:1008B000982F0E94B30A17FF06C020E030E040E8FE
:1008C00057E40E94320920E030E040E650E40E9404
:1008D0005F090E941C0BDC01CB014AE050E06BE198
:1008E00076E00E94960D0E94E60687E893E00E945B
:1008F000E60680911306909114064AE050E06BE101
:1009000076E00E94960D0E94E6068FE893E00E9432
:10091000E6068091FC038823B1F48091280690912B
:1009200029060197E1F087E487B9809161008F770C
:1009300080936100809162008F778093620082E0F3
:100940008093FC03DCC0823061F484B195B1909354
:10095000140680931306109229061092280683E04D
:10096000EFCF833009F049C082E487B9809128062F
:10097000909129060197B9F4809107069091080695
:10098000209107063091080644B155B175E03695BF
:1009900027957A95E1F7821B930B840F951F90930F
:1009A000080680930706809161008B7F8093610029
:1009B000809161008E7F80936100809162008460ED
:1009C00080936200809162008E7F809362008091AC
:1009D0006200877F80936200809162008D7F8093A8
:1009E0006200809161008860809361008091610065
:1009F00082608093610084E0A3CF8430C9F4029BBD
:100A000005C0109229061092280606C081E090E0E9
:100A10009093290680932806809162008B7F8093B3
:100A200062008091620088608093620085E088CFD8
:100A3000853009F049C083E487B9809128069091F8
:100A400029060197B9F48091170690911806209114
:100A500017063091180644B155B165E036952795D3
:100A60006A95E1F7821B930B840F951F90931806EC
:100A70008093170680916100877F80936100809149
:100A800061008D7F80936100809162008860809317
:100A90006200809162008D7F80936200809162008D
:100AA0008B7F80936200809162008E7F80936200D2
:100AB0008091610084608093610080916100816019
:100AC0008093610086E03CCF8630D1F4039B05C063
:100AD000109229061092280606C081E090E09093BB
:100AE00029068093280680916200877F80936200A8
:100AF000809162008460809362001092FC03369AB9
:100B0000FF91EF91BF91AF919F918F917F916F91E5
:100B10005F914F913F912F911F910F910F900FBEB9
:100B20000F901F9018951F920F920FB60F921124DD
:100B30002F938F939F93EF93FF939BB12CB1E091F1
:100B4000FF04EF5FEF7780910005E81711F482E072
:100B500008C0892F8871E093FF04FF27E358FB4FFB
:100B6000208380930105FF91EF919F918F912F91A9
:100B70000F900FBE0F901F9018951F920F920FB6F7
:100B80000F9211248F939F93EF93FF939091FD0405
:100B90008091FE04981761F0E091FE04EF5FEF771B
:100BA000E093FE04FF27E350FC4F80818CB901C025
:100BB0005598FF91EF919F918F910F900FBE0F90DD
:100BC0001F9018959C011092FD041092FE04109243
:100BD000FF041092000597FF03C082E08BB93F77B6
:100BE000832F99278093900029B988E98AB986E0F4
:100BF0008093950008959091FF04809100059817C7
:100C000019F480E091E00895E0910005EF5FEF773F
:100C1000E0930005FF27E358FB4F208180910105F9
:100C20009927982F8827820F911D0895282F90913A
:100C3000FD049F5F9F778091FE049817E1F3E92FF1
:100C4000FF27E350FC4F20839093FD04559A0895AD
:100C5000CF93DF93EC0103C021960E941606888192
:100C60008823D1F7DF91CF910895CF93DF93EC01E3
:100C700002C00E941606FE01219684918823C9F7BE
:100C8000DF91CF9108951F920F920FB60F9211240A
:100C90002F938F939F93EF93FF9390919B002091BD
:100CA0009C00E0910406EF5FEF7780910506E8175E
:100CB00011F482E008C0892F8871E0930406FF27B1
:100CC000EE57FA4F208380930606FF91EF919F9194
:100CD0008F912F910F900FBE0F901F9018951F921C
:100CE0000F920FB60F9211248F939F93EF93FF9360
:100CF0009091020680910306981769F0E09103062F
:100D0000EF5FEF77E0930306FF27EE5FFA4F8081F6
:100D100080939C0005C080919A008F7D80939A00FB
:100D2000FF91EF919F918F910F900FBE0F901F90A9
:100D300018959C0110920206109203061092040668
:100D40001092050697FF04C082E080939B003F77D6
:100D5000832F9927809398002093990088E98093A6
:100D60009A0086E080939D000895909104068091FA
:100D70000506981719F480E091E00895E0910506C2
:100D8000EF5FEF77E0930506FF27EE57FA4F2081DC
:100D9000809106069927982F8827820F911D089524
:100DA000282F909102069F5F9F77809103069817E6
:100DB000E1F3E92FFF27EE5FFA4F208390930206BD
:100DC00080919A00806280939A000895CF93DF9378
:100DD000EC0103C021960E94D00688818823D1F7B8
:100DE000DF91CF910895CF93DF93EC0102C00E9471
:100DF000D006FE01219684918823C9F7DF91CF9117
:100E0000089540E050E013C020E030E00000000012
:100E100000000000000000000000000000002F5F44
:100E20003F4F61E02030360789F74F5F5F4F48172B
:100E3000590751F70895BA9AB998BC9AC29AC498BA
:100E400008958BE993E00E94280684E690E00E94D2
:100E500001078FE993E00E9428068CE291E00E944E
:100E6000010787EA93E00E94280608958BE993E042
:100E70000E94280684E690E00E9401078EEA93E033
:100E80000E94280684E690E00E94010785EB93E02B
:100E90000E94280684E690E00E9401078CEB93E014
:100EA0000E94280684E690E00E94010783EC93E00C
:100EB0000E94280684E690E00E9401078AEC93E0F5
:100EC0000E94280684E690E00E94010781ED93E0ED
:100ED0000E94280684E690E00E94010788ED93E0D6
:100EE0000E94280684E690E00E9401078FE993E0C3
:100EF0000E9428068CE291E00E94010787EA93E0B5
:100F00000E94280608950F931F93182F062F8BE930
:100F100093E00E94280684E690E00E94010780EE9C
:100F200093E00E942806812F805D0E94160684EEC1
:100F300093E00E942806802F805D0E94160686EEB0
:100F400093E00E94280684E690E00E94010789EE63
:100F500093E00E9428061F910F910895EF92FF924F
:100F60000F931F937B018C0120E030E040E05FE4B1
:100F70000E947D0A88237CF020E030E040E05FE4BE
:100F8000C801B7010E9401090E941C0B605070400B
:100F90008040904804C0C801B7010E941C0B1F91FB
:100FA0000F91FF90EF900895A0E0B0E0EAEDF7E038
:100FB0000C94DF0DFC016A019081923008F41BC192
:100FC000DB018C91823080F0943061F4843009F040
:100FD00012C19181EB018981981709F40CC1E3EFEB
:100FE000F3E009C1843011F4FB0105C1823091F4B2
:100FF000923009F000C1EA01DF0188E00D9009920A
:101000008150E1F78181FB0191818923E601898388
:10101000F601F1C0923041F362807380EB018A8067
:101020009B80E480F580068117812C813D814E8173
:101030005F815301A818B908C501B7FCABC0809700
:101040000CF457C0861497040CF4BEC03401EE248F
:10105000FF2487019181FB018181981709F4A6C0C3
:10106000992309F49CC02E193F09400B510B57FDE1
:10107000B0C0E60119827B826A82F601248335833F
:1010800046835783E6012C813D814E815F81790142
:101090008A01DA01C9010197A109B1098F5F9F4F48
:1010A000AF4FBF43F8F4E6016A817B81A801970145
:1010B000220F331F441F551F6150704079018A0170
:1010C000DA01C9010197A109B1098F5F9F4FAF4FA5
:1010D000BF4360F3E6017B836A83F6012483358393
:1010E0004683578383E0D6018C9357FD39C0F601C0
:1010F00082C086149704B4F4C0E0D0E0DA01C901DC
:1011000081709070A070B07056954795379527956F
:10111000282B392B4A2B5B2B2196AC16BD0671F779
:101120008A0C9B1C681479040CF094CFC0E0D0E0CA
:101130005401A618B708D801C70181709070A0703B
:10114000B07016950795F794E794E82AF92A0A2BC8
:101150001B2B2196AC16BD0671F76A0C7B1C7ACF4F
:10116000DA01C901B695A7959795879521703070DA
:1011700040705070282B392B4A2B5B2BE6012C83B7
:101180003D834E835F838A819B8101969B838A8303
:10119000F60131C0882799278A199B0950CFE21A96
:1011A000F30A040B150BA801970161CFE60199839F
:1011B0007B826A822E0D3F1D401F511FF601248342
:1011C0003583468357838ECF20E030E040E050E007
:1011D00041CF81E0E60189837B826A825095409508
:1011E000309521953F4F4F4F5F4FF6012483358354
:1011F0004683578347CFCF01EEE0CDB7DEB70C94DF
:10120000FB0DA0E2B0E0E7E0F9E00C94E70D6983A4
:101210007A838B839C832D833E834F83588789E118
:10122000E82EF12CEC0EFD1EB701CE0101960E94B6
:101230008E0C8E010F5E1F4FB801CE0105960E94E5
:101240008E0C8A8991E089278A8BAE01475F5F4FB8
:10125000B801C7010E94D4070E946C0BE6E0A0967B
:101260000C94030EA0E2B0E0E8E3F9E00C94E70D83
:1012700069837A838B839C832D833E834F83588736
:1012800099E1E92EF12CEC0EFD1EB701CE0101967D
:101290000E948E0C8E010F5E1F4FB801CE01059685
:1012A0000E948E0CAE01475F5F4FB801C7010E94DC
:1012B000D4070E946C0BE6E0A0960C94030EA0E20B
:1012C000B0E0E5E6F9E00C94DB0D69837A838B836B
:1012D0009C832D833E834F8358878E01075E1F4F6B
:1012E000B801CE0101960E948E0CF1E1EF2EF12C97
:1012F000EC0EFD1EB701CE0105960E948E0C898D65
:10130000823078F09989923040F420E09A8D8A8971
:10131000981321E02A8BB701E9C0843051F4923050
:1013200061F020E09A8D8A89981321E02A8FB80114
:10133000DDC0943029F4823041F763EF73E0D6C00A
:10134000823079F3923009F32D8D3E8D4F8D58A167
:101350008D899E89AF89B88D222433242101AA2446
:10136000BB246501EE24FF24870160E070E00DC01E
:101370006F5F7F4F6032710599F1880F991FAA1F27
:10138000BB1F569547953795279520FF19C0280E06
:10139000391E4A1E5B1E662477244301281639062F
:1013A0004A065B0628F4E1E06E2E712C812C912C0C
:1013B000AE0CBF1CC01ED11EA60CB71CC81CD91C6D
:1013C000EE0CFF1C001F111FB7FFD2CFE1E06E2E05
:1013D000712C812C912CE628F72808291929C8CFCF
:1013E0008B8D9C8D2B893C89820F931F02969C8745
:1013F0008B871A869A8D8A89981711F081E08A87DF
:10140000D7FE17C08B859C85A0FE0CC056944794D0
:101410003794279420E030E040E050E8222A332A35
:10142000442A552AD694C794B794A79401969C87CA
:101430008B8730E0A31630E0B30630E0C30630E41B
:10144000D30618F58B859C850EC0220C331C441CDA
:10145000551C019720E0A21620E0B20620E0C2064B
:1014600020E4D20680F4AA0CBB1CCC1CDD1C57FE69
:10147000ECCF31E0632E712C812C912CA628B7285B
:10148000C828D928E2CF9C878B87D601C5018F77E2
:101490009070A070B07080349105A105B10551F035
:1014A000AD86BE86CF86D88A83E08987BE01675F16
:1014B0007F4F1CC0A7FCF4CF211431044104510418
:1014C00079F380E490E0A0E0B0E0A80EB91ECA1E57
:1014D000DB1E80E8682E8FEF782E8FEF882E8FEF3F
:1014E000982EA620B720C820D920DACFCB010E94A1
:1014F0006C0BE2E1A0960C94F70DA8E1B0E0E3E8F4
:10150000FAE00C94E70D69837A838B839C832D83A7
:101510003E834F83588781E1E82EF12CEC0EFD1EAF
:10152000B701CE0101960E948E0C8E01075F1F4FFE
:10153000B801CE0105960E948E0C8989823018F47C
:101540002FEF3FEF0BC089858230D0F3B801C70180
:101550000E942D0D282F332727FD3095C901E6E085
:1015600068960C94030EA8E0B0E0E9EBFAE00C9466
:10157000EA0D9B01AC0183E089831A8257FD51C0BB
:10158000211531054105510539F482E08983CE01E9
:1015900001960E946C0B4CC0EEE1F0E0FC83EB8303
:1015A0008A818823C9F1203010E0310710E041071B
:1015B00010E85107C9F188279927DC01821B930B9A
:1015C000A40BB50B8D839E83AF83B8872D813E819D
:1015D0004F815885203080E0380780E0480780E45C
:1015E0005807A8F6EB81FC81DA01C901880F991F21
:1015F000AA1FBB1F31979C01AD01803010E09107FD
:1016000010E0A10710E4B10778F3FC83EB838D832E
:101610009E83AF83B887BBCF2D833E834F8358878C
:10162000D5CF81E08A83ACCF60E070E080E09FECB2
:10163000E3E028960C94060EACE0B0E0E2E2FBE0BA
:101640000C94EB0D69837A838B839C83BE016B5F63
:101650007F4FCE0101960E948E0C8D81823061F009
:10166000823050F0843069F48E81882359F52FEF51
:101670003FEF4FEF5FE72AC020E030E040E050E06E
:1016800025C02F81388537FDF7CF2F31310564F71D
:101690008EE190E0821B930B29853A854B855C8512
:1016A00004C056954795379527958A95D2F78E8130
:1016B000882361F050954095309521953F4F4F4FCD
:1016C0005F4F04C020E030E040E050E8CA01B901BB
:1016D000E2E02C960C94070E4F925F926F927F92ED
:1016E0008F929F92AF92BF92DF92EF92FF920F93F1
:1016F0001F9320E030E040E050E0FC01E480F58002
:1017000006811781D1808081823038F4D801C701E9
:10171000A061AF77B0706FEFD9C0843009F46EC0AC
:10172000823009F471C0E114F1040105110509F4D6
:101730006BC0828193816FEF823896070CF06AC08C
:1017400062E87FEF681B790B6A3171050CF080C08D
:1017500047015801062E04C0B694A7949794879425
:101760000A94D2F744245524320181E090E0A0E0AD
:10177000B0E004C0880F991FAA1FBB1F6A95D2F75B
:101780000197A109B109E822F9220A231B23E114D8
:10179000F1040105110529F061E0462E512C612C60
:1017A000712C85017401E428F52806291729D80130
:1017B000C7018F779070A070B07080349105A1053B
:1017C000B10509F457C0D801C701CF96A11DB11DBD
:1017D00060E070E08030E0E09E07E0E0AE07E0E42B
:1017E000BE0710F061E070E027E0B695A7959795E9
:1017F00087952A95D1F7AF77B07068C080E090E008
:10180000A0E0B0E06FEF62C080E090E0A0E0B0E068
:1018100060E05CC0803891058CF7BC0161587F4F57
:10182000D801C7018F779070A070B0708034910597
:10183000A105B105A1F08FE390E0A0E0B0E0E80ED3
:10184000F91E0A1F1B1F17FD28C0D801C701CCCFE6
:1018500060E070E080E090E0A0E0B0E0CCCFE7FE98
:10186000F2CF80E490E0A0E0B0E0E80EF91E0A1F9D
:101870001B1FE9CFE7FC18C080E090E060E0E616AF
:1018800060E0F60660E0060760E4160710F081E00D
:1018900090E0BC01D801C701A7CF16950795F79432
:1018A000E7946F5F7F4FD1CFD801C701805C9F4F16
:1018B000AF4FBF4F60E070E08030E0E09E07E0E0B7
:1018C000AE07E0E4BE0708F48FCF8CCF282F392F66
:1018D0009A2F9F77842F8078892B962F9795992719
:1018E00097958F77482F492B6695852F8078862B83
:1018F000D794DD24D7948F77582F5D29CA01B90179
:101900001F910F91FF90EF90DF90BF90AF909F904D
:101910008F907F906F905F904F900895FC01DB0156
:10192000208131819281492F4F7750E0991F99276B
:10193000991F8381682F660F692B881F8827881F4E
:10194000FD018183662309F049C021153105410558
:10195000510509F470C082E89FEFFD0193838283F3
:10196000220F331F441F551F220F331F441F551FC3
:10197000220F331F441F551F220F331F441F551FB3
:10198000220F331F441F551F220F331F441F551FA3
:10199000220F331F441F551F83E08C932030F0E04B
:1019A0003F07F0E04F07F0E45F0790F482E89FEF15
:1019B000220F331F441F551F0197203060E0360768
:1019C00060E0460760E4560798F3FD019383828345
:1019D000FD01248335834683578308956F3F71F15A
:1019E000862F99278F579040FD019383828383E050
:1019F0008C93220F331F441F551F220F331F441F88
:101A0000551F220F331F441F551F220F331F441F22
:101A1000551F220F331F441F551F220F331F441F12
:101A2000551F220F331F441F551F506424833583D5
:101A300046835783089582E08C93089521153105DC
:101A40004105510519F484E08C93089544FD02C0CA
:101A50001C92BECF81E08C93BBCFEF92FF920F938D
:101A60001F93CF93DF93FC01DB018081823050F024
:101A70009C91923038F0843041F49430B1F08181FF
:101A8000882381F461E070E04BC09430E9F182304A
:101A9000A1F09230A1F36181ED018981681791F085
:101AA000662381F36FEF7FEF3BC0EB018981682FE5
:101AB00077278181681B710933C0923059F560E046
:101AC00070E02EC022813381ED018A819B818217D3
:101AD000930734F3281739079CF0E480F5800681DA
:101AE0001781FD0124813581468157812E153F05DF
:101AF00040075107A8F2E216F30604071507F8F6A7
:101B0000662309F0BFCFCECFFB018181882309F086
:101B1000B9CFC8CFEB018981882309F0B3CFC2CFF9
:101B2000CB01E6E0CDB7DEB70C94030EFB019F01BD
:101B3000E8944230C4F04532B4F44A3029F497FBBB
:101B40001EF4909581959F4F642F77270E94C70DB3
:101B5000805D8A330CF0895D8193CB010097A1F7FA
:101B600016F45DE251931082C9010C94B70DDC01AB
:101B7000FC0101900020E9F73297AE17BF0730F45F
:101B80007C916081708331976D93F7CF0895AA1B84
:101B9000BB1B51E107C0AA1FBB1FA617B70710F058
:101BA000A61BB70B881F991F5A95A9F7809590958A
:101BB000BC01CD0108952F923F924F925F926F9298
:101BC0007F928F929F92AF92BF92CF92DF92EF92CD
:101BD000FF920F931F93CF93DF93CDB7DEB7CA1B4E
:101BE000DB0B0FB6F894DEBF0FBECDBF09942A8879
:101BF000398848885F846E847D848C849B84AA8421
:101C0000B984C884DF80EE80FD800C811B81AA81AD
:101C1000B981CE0FD11D0FB6F894DEBF0FBECDBF78
:041C2000ED01089535
:101C2400554152543120486F7374205465737420A5
:101C34004C696E65200A0D0056616C696420636FFF
:101C44006D6D616E6473206172653A205320522079
:101C540054204C2041207564206C7220696F202B25
:101C64002D203132333435360A0D00532053657438
:101C7400726567697374657220666F72204175724C
:101C8400656C373032300A0D00522052656164723F
:101C9400656769737465722066726F6D2041757231
:101CA400656C373032300A0D005420546573746DFE
:101CB4006F64652C2073656E642032353020736147
:101CC4006D6520636861726163746572730A0D00E7
:101CD4004C204C696E65746573742061636B6E6F20
:101CE400776C656467650A0D004120416C61726D13
:101CF40020746573742061636B6E6F776C656467C1
:101D0400650A0D0075702F646F776E206C656674BC
:101D14002F7269676874207A6F6F6D20696E2F6FF8
:101D2400757420666F637573202B2F2D0A0D003197
:101D3400323334353620736176652061637475619E
:101D44006C2063616D657261706F736974696F6E25
:101D540020746F2070726573657420737461746984
:101D64006F6E20312E2E360A0D006F6E652074754D
:101D7400726E006669656C643D000A0D0020726530
:101D84006365697665642C204C696E65746573744B
:101D94002E2E6F6B0A0D0053657472656769737438
:101DA40065723A200D0A00666572746967210D0A2E
:101DB400005265616472656769737465723A200DD7
:101DC4000A00546573746D6F64653A0A0D004747E1
:101DD400474747474747474747474747474747478F
:101DE400474747474747474747474747474747477F
:101DF400474747474747474747474747474747476F
:101E0400474747474747474747474747474747475E
:101E1400474747474747474747474747474747474E
:101E2400474747474747474747474747474747473E
:101E34004747006162636465666768696A6B6C6DD5
:101E44006E6F707172737475767778797A414243E4
:101E54004445464748494A4B4C4D4E4F50515253C6
:101E64005455565758595A0A0D0073656E742074A8
:101E74006F20417572656C2C2072656164790A0D5E
:101E840000726561647920746F2073656E642064E8
:101E9400617461200D0A0052467369676E616C209B
:101EA4006C6F73740A0D0020566F6C740A0D002059
:101EB40020766F6C746167650A0D002B2B2B004133
:101EC400545331360D0A00415443430D0A00415422
:101ED40053310D0A00415453320D0A004154533317
:101EE4000D0A00415453340D0A00415453350D0A70
:101EF40000415453360D0A0041545331350D0A0044
:101F0400415453003D000D0A00415457522C4343A1
:0C1F14000D0A00000000000000000000AA
:00000001FF
